:100000000C941E060C940A280C9437280C9446066F
:100010000C9446060C9446060C9446060C94460630
:100020000C9446060C9446060C9422130C94460637
:100030000C9446060C9446060C9446060C94460610
:100040000C9464280C9446060C94522C0C94952C19
:100050000C9446060C9446060C9446060C944606F0
:100060000C9446060C9446068518E718C618C9185D
:10007000CC18CF18D218D518D818E718E118191AC3
:100080001B1A1B1A191A1B1A1B1A1B1A1B1A1B1ACA
:100090001B1A1B1A1B1A1B1A1B1A1B1A1B1A1B1AB8
:1000A0009F191B1A1B1A1B1A1B1A1B1A10191B1A31
:1000B0001B1A1B1A1B1A1B1A1B1A1B1A1B1A1B1A98
:1000C0001B1A1B1A1B1A1B1A1B1A1B1AAB19AB196A
:1000D000AB19AB19AB19AB19AB19AB19AB191B1A8F
:1000E0001B1A1B1A1B1A1B1A1B1A1019AA19AA1958
:1000F000AA19AA191B1AB819BE19C419CA19D019F4
:10010000D619DC19E219EC19F619001A0A1A511954
:1001100013191B1A1B1A1B1A1B1A9F191B1A1B1ABD
:100120001B1A1B1A1B1A1B1A1B1A1B1AA919A9190D
:10013000A919A9191B1AB819BE19C419CA19D019B5
:10014000D619DC19E219EC19F619001A0A1A511914
:1001500013191B1A1B1A1B1A1B1A9F194E1A4E1A17
:100160004E1A4E1A4E1A4E1A4E1A4E1A4E1A4E1A4F
:100170004E1A4E1A4E1A641B641B641B641B641BCC
:10018000641B931A9D1AA71AB11A0E1B181B271B62
:10019000381BC01CD51CE11CEA1CF91C1E1D271DA8
:1001A000701D391D832089208F209620A420C62011
:1001B000E420456E746572206D656E752E2E2E00DE
:1001C000546F67676C6564206D6963726F50504D42
:1001D00000546F67676C656420696E76657274653C
:1001E000642050504D2100546F67676C6564205443
:1001F00058206D7574696E672100546F67676C6570
:10020000642074656C656D65747279210050726F3D
:10021000746F636F6C206572726F72207769746897
:100220002052580054696D656F7574207768656E4B
:1002300020636F6E6E656374696E6720746F205201
:100240005800507265737320616E79206B65792058
:10025000746F2063616E63656C00436F6E6E6563DF
:1002600074696E6720746F2052582C20706F776508
:100270007220757020746865205258202877697440
:10028000682062696E6420706C7567206966206EF4
:100290006F74207573696E6720616C776179732064
:1002A00062696E642900546F67676C656420276912
:1002B0006D6D656469617465206F75747075742700
:1002C00000546F67676C65642027736C61766520E6
:1002D0006D6F64652700546F67676C6564202761E4
:1002E0006C776179732062696E642700546F676769
:1002F0006C65642050504D206368616E6E656C20A3
:100300006C696D69740053657420525353492069B8
:100310006E6A656374696F6E206368616E6E656C8A
:100320002028303D3D64697361626C652900536526
:10033000742050504D206D696E696D756D20737914
:100340006E630053657420626561636F6E20696E31
:1003500074657276616C0053657420626561636FC9
:100360006E2064656C617900536574206265616319
:100370006F6E206672657175656E637920696E2097
:10038000487A3A20303D64697361626C652C205074
:10039000783D504D52206368616E6E656C20782CFC
:1003A0002046783D465253206368616E6E656C202E
:1003B00078005365742050574D2073746F7020641B
:1003C000656C61792028302064697361626C6564B2
:1003D0002C20312D323535203D3D20302E317320FB
:1003E0002D2035306D696E29005365742050504DB5
:1003F0002073746F702064656C61792028302064EC
:10040000697361626C65642C20312D323535203D75
:100410003D20302E3173202D2035306D696E29003E
:10042000536574206661696C736166652064656CF0
:1004300061792028302064697361626C65642C20C6
:10044000312D323535203D3D20302E3173202D2089
:1004500035306D696E29002A2A2A2A2A2A2A2A2A50
:100460002A2A2A2A2A2A2A2A2A2A2A2A2A2A2A2AEC
:100470002A2A2A2A0052582041636B6564202D20C5
:1004800072657665727420737563636573736675E0
:100490006C21002A2A2A2A2A2A2A2A2A2A2A2A2AAD
:1004A0002A2A2A2A2A2A2A2A2A2A2A2A2A2A2A2AAC
:1004B000002A2A2A2A2A2A2A2A2A2A2A2A2A2A2AC6
:1004C0002A2A2A2A2A2A2A2A2A2A2A2A2A2A00528E
:1004D000582041636B6564202D20757064617465DC
:1004E000207375636365737366756C21002A2A2A0D
:1004F0002A2A2A2A2A2A2A2A2A2A2A2A2A2A2A2A5C
:100500002A2A2A2A2A2A2A2A2A2A0056616C696457
:100510002063686F69636573206172653A205B319F
:100520005D2D5B31365D20286368616E6E656C20E1
:10053000312D31362900536574206F7574707574D0
:1005400020666F7220706F727420005B585D2061AE
:10055000626F7274206368616E67657320616E6498
:10056000206578697420525820636F6E6669670051
:100570005B535D20736176652073657474696E6783
:100580007320746F205258005B525D20726576654F
:1005900072742052582073657474696E6773207486
:1005A0006F2064656661756C747300557365206EA9
:1005B000756D62657273205B312D445D20746F2010
:1005C0006564697420706F727473205B452D515D92
:1005D00020666F722073657474696E677300202DD6
:1005E00020726563656976657220636F6E66696700
:1005F000757261746F722C20727820737720000AF4
:100600000A6F70656E4C52536E67200053657420FC
:1006100073657269616C2062617564726174653AB8
:10062000200056616C69642063686F696365733A82
:100630002031202D20342B34202F2032202D203823
:10064000202F2033202D20382B34202F2034202D14
:10065000203132202F2035202D2031322B34202FF5
:100660002036202D20313600536574204368616E9A
:100670006E656C20636F6E6669673A20005365741F
:100680002044617461726174652028302D32293AEA
:10069000200053657420486F70206368616E6E653A
:1006A0006C7320286D61782032342C207365706162
:1006B000726174656420627920636F6D6D61732966
:1006C0002076616C69642076616C75657320312DCC
:1006D0003235353A2000536574206368616E6E656B
:1006E0006C2073706163696E6720287831306B48C5
:1006F0007A293A200053657420524620706F77653E
:10070000722028302D37293A200053657420524634
:10071000206D6167696320286865782920652E67E8
:100720002E20307844454144463030443A2000532E
:1007300065742062617365206672657175656E63AC
:10074000792028696E20487A293A20005B5A5D207A
:10075000656E746572207265636569766572206383
:100760006F6E66696775726174696F6E2075746902
:100770006C79005B465D20646973706C61792061FF
:10078000637475616C206672657175656E63696509
:10079000732075736564005B525D2063616C6375E3
:1007A0006C6174652072616E646F6D206B65792079
:1007B000616E6420686F70206C697374005B495DC2
:1007C000207265696E697469616C697A6520736508
:1007D0007474696E677320746F20736B65746368DB
:1007E0002064656661756C7473005B585D2072658A
:1007F00076657274206368616E67657320616E64EC
:100800002065786974206D656E75005B535D20739B
:100810006176652073657474696E677320746F20E8
:10082000454550524F4D20616E64206578697420B3
:100830006D656E7500557365206E756D62657273BA
:10084000205B302D395D20746F20656469742070E1
:100850006172616D657465727300202D2053797328
:1008600074656D20636F6E66696775726174696F18
:100870006E000A0A6F70656E4C52536E672000510D
:1008800029204F7574707574206265666F726520DB
:100890006C696E6B20283D465329203A2000502970
:1008A00020536C617665206D6F64652028657870D3
:1008B0006572696D656E74616C293A20004F29205C
:1008C00054696D65642042494E44206174207374FC
:1008D000617274757020203A20004E292050504DCE
:1008E000206F7574707574206C696D69746564200F
:1008F000202020203A200044495341424C454400E6
:100900004D292050504D205253534920746F20637D
:1009100068616E6E656C202020203A20004C2920F2
:1009200050504D206D696E696D756D2073796E63E1
:10093000202875732920203A200044495341424C15
:100940004544004B29204661696C736166652062ED
:100950006561636F6E20696E74762E2028312D32AA
:10096000353573293A20004A29204661696C736144
:10097000666520626561636F6E2064656C617920D5
:1009800028302D323535203D3E20313073202D204A
:100990003135306D696E293A200049292046616958
:1009A0006C7361666520626561636F6E206672714B
:1009B0002E203A200048292050574D2073746F7024
:1009C0002064656C6179202020202020203A2000BE
:1009D00047292050504D2073746F702064656C61FE
:1009E00079202020202020203A200046292046611E
:1009F000696C736166652064656C617920202020D4
:100A00002020203A200050574D206368616E6E65AB
:100A10006C200066756E6374696F6E3A2000292041
:100A2000706F72742000506F776572546F776572C3
:100A300000445446205548462033322D62697420C4
:100A400031306368004F70656E4C52536E67525878
:100A5000206D696E6920342F36636800466C7974A6
:100A6000726F6E2F4F72616E6765525820554846FF
:100A70002038636800525820747970653A20004429
:100A8000697361626C656400487A00203D3D200016
:100A900043616C63756C61746564207061636B6540
:100AA0007420696E74657276616C3A200042292068
:100AB0004D6963726F202868616C66292050504D23
:100AC000202020203A00412920496E766572746505
:100AD000642050504D20696E20202020203A0030A4
:100AE00029204D7574652062757A7A657220286DAB
:100AF0006F73746C79293A003929205365726961E2
:100B00006C2062617564726174653A00736D617224
:100B100074506F7274004672536B79005472616E38
:100B200073706172656E740044697361626C6564B0
:100B30000038292054656C656D657472793A2020FF
:100B40002020202020003729204368616E6E656CCC
:100B500020636F6E6669673A202000362920446161
:100B60007461726174652028302D32293A2020206A
:100B700000352920486F70206368616E6E656C7364
:100B80003A2020202020003429204368616E6E65C1
:100B90006C2073706163696E673A202000332920EE
:100BA000524620706F7765722028302D37293A2001
:100BB0002020003229205246206D616769633A2067
:100BC0002020202020202020003129204261736530
:100BD000206672657175656E63793A202020000089
:100BE00000000700020100000304060000000000EE
:100BF00000000001020408102040800102040810D7
:100C00002001020408102004040404040404040263
:100C10000202020202030303030303000000002395
:100C2000002600290000000000250028002B0000FD
:100C3000000000240027002A0000832D11241FBE7D
:100C4000CFEFD8E0DEBFCDBF13E0A0E0B1E0E4E13C
:100C5000F1E602C005900D92A83CB107D9F716E065
:100C6000A8ECB3E001C01D92AE38B107E1F71CE07B
:100C7000CCE3DCE004C02297FE010E948C2ECA3334
:100C8000D107C9F70E94BF2D0C9488300C94000046
:100C900080917305813019F482E08093730580910F
:100CA0007305833019F484E0809373050895A89543
:100CB0000895DC01ED91FC910190F081E02D099502
:100CC00008952091740530917505382748E0C901D1
:100CD000880F991F37FF06C09C0151E2252750E17C
:100CE000352701C09C01415091F730937505209341
:100CF0007405089588E38093760580E092ECA1E086
:100D0000B0E08093770590937805A0937905B09330
:100D10007A0587E08093830580E091EAACEBB3E34A
:100D200080937B0590937C05A0937D05B0937E0511
:100D300085E0809384058DEE9EEFADEABEED809355
:100D40007F0590938005A0938105B0938205E5E827
:100D5000F5E080E090E0863028F4DC01AE54BC4F32
:100D60002C9101C020E0219301968831910599F7DB
:100D700082E080939D058AE080939E05089580E03F
:100D80009EECADEEB4E38093BB059093BC05A093BD
:100D9000BD05B093BE0580E090E0A0E0B0E5809393
:100DA000BF059093C005A093C105B093C205E3ECC5
:100DB000F5E080E081938F5F8031E1F70895A0E056
:100DC000B0E0E5EEF6E00C94552ED82F0E94BA283C
:100DD0006115710581059105C9F30E94F82E1092E5
:100DE0007F05109280051092810510928205C4E063
:100DF000812C912C54018A94C0907F05D09080055D
:100E0000E0908105F0908205FE2CED2CDC2CCC24AA
:100E10000E94F32EA50194010E94342E6C0D7D1DBD
:100E20008E1D9F1D60937F057093800580938105C3
:100E300090938205C15001F7DD2309F450C005E805
:100E400015E0E801A12CB12C62E3C62ED12CE12CD7
:100E5000F12C8881882309F442C0B39419F40E94CC
:100E60007A063DC00E94F32EA70196010E94342EFF
:100E7000E1E0E60FA5E8B5E08A2F801B8A1520F493
:100E80008D918E13F9CFE9CF2091840530E0A0E158
:100E9000B7E20E94CC2D9B01AC01AE2FB0E00E94C6
:100EA000DB2D40907B0550907C0560907D05709017
:100EB0007E05640D751D861D971D4090BB055090E5
:100EC000BC056090BD057090BE05461657066806C5
:100ED000790618F2E993A39488E1A812BACFCDB7A6
:100EE000DEB7E0E10C94712E8436910520F4BC014C
:100EF00080E090E017C09C018E3B910528F42A55B4
:100F00003109AAE0B0E00CC0823D910528F4245BD1
:100F10003109A4E6B0E004C02D5C3109A8E5B2E0D7
:100F20000E94CC2DA4E6B0E09B01AC010E94DB2D19
:100F3000089590E08C599F4F0E947407089561E0D6
:100F400086E00E94672960E086E00E94A02982E096
:100F50008093B00085E08093B10061E083E00E945F
:100F6000672960E083E00E94A0290895CF93DF9372
:100F7000EC010097E9F061E086E00E94A0299E0163
:100F800040E050E068E478EE81E090E00E94342E8A
:100F90002F3F31054105510529F020F02FEF30E0BA
:100FA00040E050E02093B3008091B000806107C022
:100FB00060E086E00E94A0298091B0008F7E80933F
:100FC000B000DF91CF91089560E08EE00E94672924
:100FD00061E08FE00E94672961E080E10E9467295B
:100FE00060E082E00E94672961E084E00E94672956
:100FF000089542E050E068E476E080E00E94EA274D
:101000000895E3E0F0E089E080935700E491E67012
:1010100081E0E63009F080E00895CF93DF93C82F98
:101020000E940108882381F0DFB781E08093720578
:10103000F8940E94570688E180936000C093600096
:10104000C1110E945706DFBFDF91CF9108958F92A3
:101050009F92AF92BF92CF92DF92EF92FF92CF9387
:10106000FC01C0A5EC2FE770F0E0E658FC4FA08132
:10107000B0E0C7FF03C024E130E002C02FE030E061
:10108000FC0197A183E1989FF0011124E25CFE4FDF
:1010900080809180A280B380A20FB31F20E43FE143
:1010A0004DE750E00E94E62DA50194010E94122E0A
:1010B0008C2F887149F469017A01E0EDCE0EE7E0EA
:1010C000DE1EE11CF11C1BC0C7FF05C060E47AE80E
:1010D0008CE29EE004C060E07EEE8AEB9BE069015A
:1010E0007A01F8EBCF0EFBE0DF1EE11CF11CA5013D
:1010F00094010E94122EC20ED31EE41EF51EC701DB
:10110000B60169517C4F8F4F9F4F28EE33E040E08E
:1011100050E00E94122EA8EEB3E00E94DB2DCF918A
:10112000FF90EF90DF90CF90BF90AF909F908F9007
:1011300008958F3F910551F048F0811522E0920704
:1011400038F08115934030F482E0089580E00895EE
:1011500081E0089583E00895A0E0B0E0E2EBF8E0DC
:101160000C945E2EEB018A01B82FB695A0E0288181
:101170003981F80120832A813B8121832C813D81A3
:1011800022832E813F812383688179814A815B811B
:101190002C813D81EE81FF819F2F9295990F990FB0
:1011A000907C272F2370922B252F2370220F220F44
:1011B000922B232F23702295207F922BF80194836A
:1011C0000B5F1F4F2896AF5FBA1788F680FF24C0C9
:1011D000888199810E949908D82E8A819B810E94DA
:1011E0009908E82E8C819D810E949908F82E8E81A5
:1011F0009F810E949908F0E4DF9EA001112490E1F4
:10120000E99E90011124242B282BE4E0FE9EB001DE
:101210001124262BF8012083CDB7DEB7E7E00C942C
:101220007A2E803223E0920708F1883E23E092076D
:1012300040F48F519340E4E096958795EA95E1F765
:101240000895803D27E0920718F48C5D934008953F
:10125000883928E0920768F4885C974074E0969596
:1012600087957A95E1F78D509C4F089580E090E046
:1012700008958FEF93E008958C30910540F4A4E039
:10128000880F991FAA95E1F7885D9C4F0895843FC8
:1012900023E0920718F484529C4F0895811524E0AE
:1012A000920740F48657934FF4E0880F991FFA9500
:1012B000E1F7089580E998E008959C013695279517
:1012C00025753575821B930B9C012373337396959B
:1012D00087959695879583739373820F931F9C01CF
:1012E00054E0369527955A95E1F7280F391F2F704E
:1012F0003F7041E051E0249FC001259F900D349F35
:10130000900D1124892F08954298882319F0000028
:10131000419A02C0000041980000429A00000895DE
:10132000429A000086B14298000081700895CF93E0
:10133000DF93D82F5C9A42985C98C8E08D2F807814
:101340000E948409DD0FC150C9F74298DF91CF9107
:1013500008958F770E9497090895CF93DF93D82F30
:10136000C8E08D2F80780E948409DD0FC150C9F735
:101370004298DF91CF910895CF93DF934298C8E0D0
:1013800080E0D82FDD0F0E9490098D0FC150C9F762
:10139000DF91CF9108950E94A9090E94BC095C9A2F
:1013A0000895A1E0B0E0E7EDF9E00C94632E8068C9
:1013B00069830E9497096981862F0E94AD095C9A12
:1013C0002196E2E00C947F2ECF93C0917F05C82731
:1013D000E82FF0E0EA58FA4F678589E70E94D109C3
:1013E0006C2F8DE30E94D1096C2F82E40E94D109F9
:1013F000CF91089586E20E94CB090895CF93DF93A1
:10140000EC016C818CE10E94D1096D818DE10E941B
:10141000D1096E818EE10E94D1096F8180E20E9424
:10142000D109688581E20E94D109698582E20E9422
:10143000D1096A8583E20E94D1096B8584E20E940A
:10144000D1096C8585E20E94D1096D858AE20E94EE
:10145000D1096E858EE60E94D1096F858FE60E94C4
:10146000D109688980E70E94D109698981E70E94D2
:10147000D1096A8982E70E94D109DF91CF9108954D
:10148000CF92DF92EF92FF92CF93DF936B017C01BB
:10149000C11488E3D8068CE9E8068CE1F80628F543
:1014A000C701B60120E836E948E950E00E94122E53
:1014B000E901689760E879E687E69FEF0E94EE2DE4
:1014C0006C0D7D1D8E1D9F1DF2E0660F771F881F1E
:1014D000991FFA95D1F721E732E040E050E00E94F1
:1014E000122EF22EE32E80E421C0C701B60120E0C7
:1014F0003DE241E351E00E94122EE901689760E06D
:1015000073ED8EEC9EEF0E94EE2D6C0D7D1D8E1DF9
:101510009F1D660F771F881F991F21E732E040E06B
:1015200050E00E94122EF22EE32E80E66C2F6F7197
:10153000680F85E70E94D1096E2D86E70E94D109C8
:101540006F2D87E70E94D109DF91CF91FF90EF9037
:10155000DF90CF900895682F8DE60E94D1090895FD
:101560008F929F92AF92BF92CF92DF92EF92FF92B3
:10157000CF93DF93D82F83E00E94CB09809371052E
:1015800084E00E94CB098093700560E086E00E94B1
:10159000D10961E087E00E94D1096FE789E00E94EC
:1015A000D10965E08AE00E94D10962E18BE00E94E6
:1015B000D10965E18CE00E94D1096DEF8DE00E94B8
:1015C000D10960E08EE00E94D109DD2319F08BE2A1
:1015D00091E008C020919D0533E1239FC0011124B3
:1015E000825C9E4F0E94FE096CE880E30E94D10954
:1015F0006FE082E30E94D10962E483E30E94D10993
:1016000080919E0587FF02C064E101C06AE084E327
:101610000E94D1096AE285E30E94D1096DE286E366
:101620000E94D10964ED87E30E94D10960E088E35C
:101630000E94D10960E089E30E94D109D11109C05B
:10164000C0907F05D0908005E0908105F0908205E4
:1016500007C0C5E9CC2EC1ECDC2EED2CCEEDFC2E66
:10166000CAE38F2C9924AA24BB24682D8C2F0E94B6
:10167000D109682D85E08C0F0E94D109FE2CED2C3C
:10168000DC2CCC24CF5FCE3361F76FEF83E40E9474
:10169000D1096FEF84E40E94D1096FEF85E40E94C5
:1016A000D1096FEF86E40E94D109DD2311F066E0D5
:1016B00002C0609183058DE60E94D10960E089E750
:1016C0000E94D109609184058AE70E94D10960E0F7
:1016D00083E70E94D10960E084E70E94D109D1111B
:1016E00009C060917B0570917C0580917D0590918A
:1016F0007E0504C060E071EA8CEB93E30E94400A2F
:10170000DF91CF91FF90EF90DF90CF90BF90AF909F
:101710009F908F90089561E087E00E94D10964E274
:101720008EE70E94D10963E088E00E94D10960E061
:1017300088E00E94D10965E087E00E94D10962E05B
:1017400085E00E94D10983E00E94CB098093710556
:1017500084E00E94CB0980937005089583E00E9485
:10176000CB098093710584E00E94CB0980937005BA
:1017700061E087E00E94D1096AE070E080E090E0DB
:101780000E94DD280E948B0B00000895CF92DF920B
:10179000FF920F931F93CF93DF931F92CDB7DEB7C6
:1017A000082F162F8EE399830E94D109F02EC02EA8
:1017B0009981D92E8C2D8F19811738F4F6016191FA
:1017C0006F018FE70E94D109F5CF64E085E00E94A8
:1017D000D10983E00E94CB098093710584E00E94C7
:1017E000CB09809370050E94BA2860936C057093B2
:1017F0006D0580936E0590936F0569E087E00E9408
:10180000D10981E0809373050F90DF91CF911F91F3
:101810000F91FF90DF90CF9008950F931F930E9438
:10182000C60B80917305813099F40E94BA2800910B
:101830006C0510916D0520916E0530916F05601B50
:10184000710B820B930B603A76488140910548F307
:1018500080917305813031F46EE971E082EE95E09C
:101860000E94A62A1F910F9108950F931F938091B4
:101870007305823021F41092730581E020C08091BD
:1018800073058130D9F40E94BA2800916C0510913B
:101890006D0520916E0530916F05601B710B820BF9
:1018A000930B613A76488140910540F061E087E012
:1018B0000E94D1091092730582E001C080E01F915F
:1018C0000F910895CF93DF93EC014AE050E06D2F24
:1018D00070E082EE95E00E94742B6EE282EE95E05D
:1018E0000E94782ABE0184E0769567958A95E1F793
:1018F0006F7077274AE050E082EE95E00E94742BEB
:101900006EE282EE95E00E94782ABE016F70772722
:101910004AE050E082EE95E00E94742BDF91CF9177
:101920000895D82FC0E0CD1790F4439A299A64E621
:1019300070E080E090E00E94DD284398299864E6FA
:1019400070E080E090E00E94DD28CF5FECCF6CE299
:1019500071E080E090E00E94DD28E4CF0F931F93B8
:10196000CF93DF93EC01062F15E0115051F0CE011B
:101970000E946F30081741F0602FCE010E9477302F
:10198000F4CF82E00E94910CDF91CF911F910F91D3
:101990000895A0E0B0E0EFECFCE00C94552E482E4A
:1019A000562EC0E0D0E0612C712CE12CF12C00E02F
:1019B00010E041100CC06090D40586E4689E3001B0
:1019C000112459E1E52EF12C0AEB15E01EC091E03F
:1019D00049120FC06090D405E6E46E9E30011124D8
:1019E000FBE16F0E711C49E2E42EF12C06E715E0D5
:1019F0000CC082E0481209C028E1622E772473945B
:101A0000EE24E394F12C03ED15E043018C0E9D1EB2
:101A100010927505109274053401A62CA818B12CEB
:101A2000C30101966C01AE14BF04A8F4A00EB11E50
:101A3000511006C0C3010E946F30F501808305C0BC
:101A4000F5016081C3010E94AE0CF50180810E9406
:101A500061063601E2CFC301511018C0C3010E94D4
:101A60006F30B82EC6010E946F302B2D30E0322F20
:101A70002227282B80917405909175058217930772
:101A800079F4C0E0D0E05524539493CF36016091AF
:101A900075050E94AE0C60917405C6010E94AE0CE3
:101AA000C05EDE4FC13E92E0D90708F482CF852D9B
:101AB000CDB7DEB7E0E10C94712E61E082E00E94C8
:101AC000C90C089560E082E00E94C90C8091D305A2
:101AD000853020F01092D3050E945D0D8091D305D2
:101AE0008093D405089561E080E00E94C90C61E014
:101AF00081E00E94C90C089560E080E00E94C90C5A
:101B0000882351F060E081E00E94C90C882321F015
:101B100080917605883349F00E94BF060E947A06BC
:101B200081E00E94DF060E94730D0895882319F05A
:101B30006AEA71E002C06EEA71E082EE95E00E940E
:101B4000A62A0895FF920F931F93CF93DF9369EC1A
:101B50007BE082EE95E00E94522A40917B055091F5
:101B60007C0560917D0570917E052AE030E082EE73
:101B700095E00E947B2B63EB7BE082EE95E00E9478
:101B8000522A40917F0550918005609181057091A6
:101B9000820520E130E082EE95E00E947B2B6DE92A
:101BA0007BE082EE95E00E94522A4AE050E060918C
:101BB000830582EE95E00E94A32B67E87BE082EE2E
:101BC00095E00E94522A4AE050E06091840582EE3E
:101BD00095E00E94A32B61E77BE082EE95E00E94F6
:101BE000522AC5E8D5E0F12C8E0188818823A9F01E
:101BF000FF2031F061EB71E082EE95E00E94752AE2
:101C000021964AE050E0F801608182EE95E00E9462
:101C10006C2BF394F8E1FF12E7CF82EE95E00E947F
:101C2000802A6BE57BE082EE95E00E94522A4AE032
:101C300050E060919D0582EE95E00E94A32B66E442
:101C40007BE082EE95E00E94522AE0919E05E770CB
:101C5000F0E0EE0FFF1FEE57FC4F6081718182EEC6
:101C600095E00E94A62A61E37BE082EE95E00E9467
:101C7000522A80919E058871883069F028F481117C
:101C800013C068E27BE00CC0803141F0883161F420
:101C90006CE07BE005C06CE17BE002C066E17BE0CC
:101CA00082EE95E00E94942A68EF7AE082EE95E059
:101CB0000E94522A409177055091780560917905EC
:101CC00070917A052AE030E082EE95E00E947B2B4D
:101CD0006FED7AE082EE95E00E94522A8091BF0576
:101CE00080710E94960D66EC7AE082EE95E00E948B
:101CF000522A8091BF0580740E94960D6DEA7AE0A9
:101D000082EE95E00E94522A8091BF0580720E9467
:101D1000960D60E97AE082EE95E00E94522A86E70D
:101D200095E00E942708AB01BC012AE030E082EE7A
:101D300095E00E945D2B6BE87AE082EE95E00E94D0
:101D4000522A86E795E00E9427089B01AC0160E4D7
:101D500072E48FE090E00E94122EBA01A9012AE0FD
:101D600030E082EE95E00E945D2B68E87AE082EE3A
:101D700095E00E94942ACDB7DEB7E5E00C947C2E66
:101D80008F929F92AF92BF92CF92DF92EF92FF928B
:101D9000811107C06FE77AE082EE95E00E94942AF5
:101DA0002FC090E00E94740724E630E040E050E04D
:101DB0000E94122ECA01B9012AE030E040E050E052
:101DC0000E94122E49015A016B017C012AE030E089
:101DD000B501A40182EE95E00E945D2B6EE282EED9
:101DE00095E00E94782A2AE030E0B701A60182EE51
:101DF00095E00E945D2B63E782EE95E00E94B82A91
:101E0000FF90EF90DF90CF90BF90AF909F908F901A
:101E100008951F93CF93DF9365E77AE082EE95E014
:101E20000E94522A80919F05813041F46CE57AE04E
:101E300082EE95E00E94942A10E050C0823019F49E
:101E400065E47AE0F5CF843019F461E37AE0F0CF0D
:101E5000853091F766E27AE0EBCFC12FD0E0C93050
:101E6000D1050CF441C068E3610F82EE95E00E9459
:101E7000782A6EE17AE082EE95E00E94522ABE0155
:101E80006F5F7F4F4AE050E082EE95E00E943C2B6E
:101E900063E17AE082EE95E00E94522AC156DA4F61
:101EA000E981E03218F566E07AE082EE95E00E9482
:101EB000522A8981803130F06DE673E082EE95E040
:101EC0000E94752A69816F7070E06F5F7F4F4AE0F2
:101ED00050E082EE95E00E94452B1F5F80914805FF
:101EE000181708F4BACF0FC061E3BECFEF70F0E06F
:101EF000EE0FFF1FEE56FC4F6081718182EE95E080
:101F00000E94A62AEACF6BEE79E082EE95E00E946D
:101F1000522A8091B7050E94C00E60ED79E082EEF2
:101F200095E00E94522A8091B8050E94C00E65EB90
:101F300079E082EE95E00E94522A8091B9050E94D4
:101F4000C00E6AE979E082EE95E00E94522A409143
:101F5000AF055091B0056091B1057091B205411582
:101F600051056105710539F12AE030E082EE95E016
:101F70000E947B2B67E679E082EE95E00E94522A70
:101F80008091B3050E949907AB01BC012AE030E0C3
:101F900082EE95E00E947B2B63E479E082EE95E08F
:101FA0000E94522A4AE050E06091B40582EE95E02A
:101FB0000E94A32B06C06AE379E082EE95E00E94BE
:101FC000942A6DE179E082EE95E00E94522A6091B8
:101FD000B5057091B6054AE050E082EE95E00E94AA
:101FE0008D2B60E079E082EE95E00E94522A6091AC
:101FF000AE05603450F470E06F5F7F4F4AE050E010
:1020000082EE95E00E94452B06C067EF78E082EEF5
:1020100095E00E94942A6AED78E082EE95E00E94B5
:10202000522A8091AD0580FF03C063EB71E002C0CE
:1020300067EB71E082EE95E00E94A62A6DEB78E0F6
:1020400082EE95E00E94522A8091AD0582700E9436
:10205000960D6EE978E082EE95E00E94522A80911A
:10206000AD0584700E94960D6FE778E082EE95E0F2
:102070000E94522A8091AD0588700E94960DDF91D2
:10208000CF911F9108950F931F93CF93DF932091CA
:1020900045052F3FA9F56FEF75E082EE95E00E94B0
:1020A000522A82E893E00E94620C6EED75E082EEA7
:1020B00095E00E94522A80914605909147050E9422
:1020C000620C6BEA75E082EE95E00E94942A68E863
:1020D00075E082EE95E00E94942A60E775E082EE5A
:1020E00095E00E94942A6BE475E082EE95E00E94F0
:1020F000942A82EE95E00E94802A0E94090F68C00F
:1021000012160CF065C0332727FD309580914805E5
:1021100090E0821793070CF45BC066E375E082EEF3
:1021200095E00E94522A60914505772767FD7095DA
:102130004AE050E082EE95E00E94452B6BE075E0AE
:1021400082EE95E00E94522A10E008E28091490553
:102150001817D0F5C12FD0E0CC0FDD1FC65BDA4FCA
:10216000288130E080914505992787FD909501975A
:102170002817390739F56BEB71E082EE95E00E9484
:10218000752A4AE050E0602F82EE95E00E946C2BA9
:102190006FEB71E082EE95E00E94752AE981EF70A5
:1021A000F0E0EE0FFF1FEE56FC4F6081718182EE72
:1021B00095E00E94752A63EC71E082EE95E00E9442
:1021C000752A0F5F1F5FC2CF82EE95E00E94802AC2
:1021D000DF91CF911F910F910895FF920F931F935D
:1021E000CF93DF93C5E8D5E0F12C8E018881882359
:1021F000D1F165EC71E082EE95E00E94752A4AE02B
:1022000050E06F2D82EE95E00E946C2B62ED71E044
:1022100082EE95E00E94752A2196F801208130E037
:10222000A0E1B7E20E94CC2D9B01AC01A0918405F6
:10223000B0E00E94DB2DAB01BC0180917B05909149
:102240007C05A0917D05B0917E05480F591F6A1F3E
:102250007B1F2AE030E082EE95E00E947B2BF39416
:10226000F8E1FF12C2CFCDB7DEB7E5E00C947C2ECB
:102270001092DF0485E6E0EEF4E0DF011D928A951E
:10228000E9F70895CF93C82F8F3719F0883009F0F8
:1022900045C0E091DF04EE23D9F1E150E093DF0483
:1022A000F0E0E052FB4F10826DE070E082EE95E0CE
:1022B0000E945906C0E08091DF04C81760F4EC2F3B
:1022C000F0E0E052FB4F608170E082EE95E00E940A
:1022D0005906CF5FF0CF60E270E082EE95E00E9499
:1022E00059066DE070E082EE95E00E945906C0E06C
:1022F0008091DF04C81778F5EC2FF0E0E052FB4F37
:10230000608170E082EE95E00E945906CF5FF0CFC9
:1023100067E082EE95E00E94782A1DC08B3119F4A7
:102320000E9438111AC08D30C1F08A30B1F080910E
:10233000DF04843668F76C2F70E082EE95E00E942F
:102340005906E091DF0481E08E0F8093DF04F0E016
:10235000E052FB4FC08380E001C081E0CF9108953F
:10236000CF93C82F0E94BA286093C8047093C90401
:102370008093CA049093CB04C093DD04CC2329F04E
:1023800040E051EE60E070E004C040E855E260E0FB
:1023900070E082EE95E00E94022DCF910895909119
:1023A000CC04492F4F7050E0BA016F5F7F4F292F47
:1023B00030E0E4E035952795EA95E1F76217730779
:1023C00059F0FA01E353FB4F808381E0890F8F704E
:1023D000907F892B8093CC0408956EE770E082EEA5
:1023E00095E00E9459060895A3E1B1E0EAEFF1E11A
:1023F0000C94562EE5E8F5E0712C8191882321F0AC
:10240000739428E17212F9CF66ED71E082EE95E0E7
:102410000E94A62A4AE050E0672D82EE95E00E94D5
:10242000A32B80E00E94B00A0E948B0B8E010E5FEE
:102430001F4FC12CD12C7601C39466246A945C2C66
:102440000E94AE284B015C012091840530E0A0E1A0
:10245000B7E20E94CC2D9B01AC01C701B6010E94DE
:10246000EE2D20917B0530917C0540917D055091AA
:102470007E05620F731F841F951F2091BB0530914D
:10248000BC054091BD055091BE052617370748078A
:10249000590718F4F80160822AC08C2D0E94E409C3
:1024A00061E070E080E090E00E94DD28F801108299
:1024B0000E94AE28681979098A099B09643F714016
:1024C0008105910540F40E94FA09F801908198175E
:1024D00078F78083EDCF85B150FE05C08B7D85B93F
:1024E000439A299A04C0846285B9439829982FEFAA
:1024F000C21AD20AE20AF20A0F5F1F4F8FEFC81604
:10250000D104E104F10409F09ACFCE019395FC01C6
:10251000D82E7FEF68EC2E2F281B271510F051E0E6
:1025200056C0DE01129651E02FEF41E03D91321787
:1025300010F0322F01C0452F5F5F5F3F11F0232F56
:10254000F5CF4193242F30E0A1E0B0E0AC0FBD1FE8
:10255000A20FB31F5C93413079F0DE01A20FB31FCD
:102560005C93423049F0AFEFBFEFAC0FBD1FA20F3D
:10257000B31F6C934E3F78F6A2E0B0E0AC0FBD1FE6
:10258000A20FB31F7C934D3F30F6A3E0B0E0AC0F39
:10259000BD1FA20FB31F6C93BECF452F242F30E079
:1025A000FC01E20FF31F6081AFEFB0E0AC0FBD1F85
:1025B000A20FB31F2C91621748F44150DC01A40F05
:1025C000B11D2C9120836C934111E8CF5F5F5715AB
:1025D00020F3372D369520E0231770F4DC01A20F8D
:1025E000B11D4C91522F530FFC01E50FF11D50818D
:1025F0005C9340832E5FF0CFF5E8EF2EF5E0FF2EE1
:102600008C01802F8D19871598F4F801C1908F01E6
:102610004AE050E06C2D82EE95E00E946C2B6CE25B
:1026200082EE95E00E94782AF701C1927F01E9CFFE
:1026300082EE95E00E94802A81E0CD5EDE4FEFE0E1
:102640000C94722E1F920F920FB60F9211241F93AB
:102650002F933F934F935F936F937F938F939F93AA
:10266000AF93BF93CF93DF93EF93FF93C091860017
:10267000D091870080918704909188042091A904CB
:10268000211155C09E01281B390B8091BF059091E7
:10269000C005A091C105B091C20585FD02C0369567
:1026A0002795253C49E03407B8F140910A0150E0F4
:1026B00060E070E02CE1B695A795979587952A95EF
:1026C000D1F70097A105B10521F481E090E0A0E0E9
:1026D000B0E084179507A607B707D8F480910A01E0
:1026E0008F3FB9F040E080910A01481780F4842FB1
:1026F00090E0880F991FFC01E757FB4F2081318143
:10270000FC01E55FFE4F318320834F5FECCF1092D9
:10271000AA0410920A010BC02D3B82E0380720F07A
:1027200080910A018031D8F08FEF80930A01D09315
:102730008804C0938704FF91EF91DF91CF91BF91FF
:10274000AF919F918F917F916F915F914F913F9149
:102750002F911F910F900FBE0F901F901895109101
:102760000A0181E0810F80930A01C9010E941109C9
:10277000E12FF0E0EE0FFF1FE757FB4F91838083BF
:10278000D6CF83E0809380008AE980938100809196
:10279000BF0586FD05C08091810080648093810023
:1027A0008FEF9FEF909389008093880080916F0056
:1027B000806280936F0008950E94620D8091D4051D
:1027C000843011F41092D40508956F3018F0869576
:1027D0008058089589E0689F802D11240895A0E015
:1027E000B0E0E5EFF3E10C945D2EC82F0E94BA280B
:1027F000009138041091390420913A0430913B043F
:102800006B017C01C01AD10AE20AF30A9701860122
:1028100049E8C41643E1D406E104F10410F0109233
:102820003C04609338047093390480933A04909385
:102830003B042091A9048FEF820F8230D8F5E091FC
:102840003C04EE2309F44EC1E13011F482E0B8C13A
:10285000E03108F034C181E08E0F80933C04F0E059
:10286000E757FB4FC083803109F0ACC1EBE8F4E0DF
:10287000213029F4A181A695A695808108C0808188
:102880009181A92FA695A695A69596958795A03195
:1028900048F4B0E090E0AA0FBB1FA55FBE4F1196B1
:1028A0009C938E931092AA04329684E0E939F8073B
:1028B000F9F688C1233009F005C1E0913C04E1112B
:1028C00004C0CF3009F07EC10DC1E83148F481E089
:1028D0008E0F80933C04F0E0E857FB4FC08372C139
:1028E000E83109F0ECC0C111EAC040E050E0ABE0D3
:1028F000CA01B3E0880F991FBA95E1F7A49F900130
:10290000A59F300D1124F901E757FB4F6081E1814C
:102910007E2F777075956795FC01EE0FFF1FE55FC1
:10292000FE4F71836083F901E657FB4FB081B69586
:10293000B695B695E181FE2FF295FF0FF07E6F2FD1
:102940006B2BE695E695E6957E2F777075956795E6
:10295000FC01EE0FFF1FE35FFE4F71836083F901FF
:10296000E557FB4FB081B295B695B695B370C1816E
:10297000DC2FDD0FDD0F6D2F6B2BC295C695C69535
:10298000C370E281E170EE0FEE0F7E2F7C2B759508
:102990006795FC01EE0FFF1FE15FFE4F71836083BF
:1029A000F901E357FB4FB081B695E181FE2FF79512
:1029B000FF27F7956F2F6B2BE6957E2F7770759518
:1029C0006795FC01EE0FFF1FEF5EFE4F7183608382
:1029D000F901E257FB4FB081B295BF70E181FE2F44
:1029E000F295F07F6F2F6B2BE295EF707E2F777053
:1029F00075956795FC01EE0FFF1FED5EFE4F71832D
:102A00006083F901E157FB4FB081BB1FBB27BB1FA0
:102A1000C181DC2FDD0F6D2F6B2BCC1FCC27CC1F82
:102A2000E281E370EE0F7E2F7C2B75956795FC019C
:102A3000EE0FFF1FEB5EFE4F71836083F901EF56CF
:102A4000FB4FB081B695B695E181FE2FF295FF0F51
:102A5000FF0FF07C6F2F6B2BE695E6957E2F77703E
:102A600075956795FC01EE0FFF1FE95EFE4F7183C0
:102A70006083F901EE56FB4F208122952695277041
:102A80003181E32FEE0FEE0FEE0F6E2F622B732FBF
:102A900072957695777075956795FC01EE0FFF1F1F
:102AA000E75EFE4F718360834F5F5F4F4230510599
:102AB00009F01ECF80919F0483FF1092AA04109208
:102AC0003C0480C0243009F07DC060913C04611159
:102AD0000BC0C83AB1F4109275051092740588EADB
:102AE0000E94610681E06CC0613019F4C093370424
:102AF00004C0623031F4C09336048C2F0E9461060A
:102B00005AC0E09136042E2F30E0220F331F462F9B
:102B100050E0C9010296841795073CF0633268F7CC
:102B2000FA01EA57FB4FC083E8CF2D5F3F4F8C2F50
:102B300090E060917405709175054217530749F450
:102B4000982F88278627972790937505809374057B
:102B500032C06817790769F580913704813049F5EB
:102B6000E13118F080E180933604F0903604CAE831
:102B7000D4E000E010E00F15D0F4FE013197808121
:102B800090E0982F88272881822B63E0969587957F
:102B90006A95E1F70E941109F801EE0FFF1FE55F4A
:102BA000FE4F918380830F5F1F4F2296E4CF1092D8
:102BB000AA0410923C0480913C04882319F08F5F92
:102BC00080933C04CDB7DEB7E8E00C94792EE82F73
:102BD000F0E0E654FA4FE185E03150F4F894F0E08B
:102BE000EE0FFF1FE55FFE4F80819181789408957D
:102BF000E03121F0E13131F483E101C082E10E9452
:102C0000FC29089580E092E00895A2E2B0E0EBE0B4
:102C1000F6E10C94532E9E012F5F3F4F80E1D901C6
:102C20001D928A95E9F764E072E082EE95E029A3AF
:102C30003AA30E94A62A0E94AE0B1D8A1E8A1F8AF2
:102C4000188E312C212C00E0812C912C5401412C28
:102C500074E7572E7BE8672E72E3772EE0E5CE2EE1
:102C6000E3ECDE2EE12CF12C84EF91E0A0E0B0E06B
:102C70008D8F9E8FAF8FB8A380E09EECADEEB4E356
:102C8000898F9A8FAB8FBC8F80E094E7ABE8B2E37B
:102C9000898B9A8BAB8BBC8B82EE95E00E94BA2B12
:102CA000892B09F4E1C082EE95E00E94E72B9C019C
:102CB00033272C32310509F442C0ACF423323105FC
:102CC00009F0ABC019821A821B821C821D821E82EF
:102CD0001F82188619861A861B861C861D861E86EC
:102CE0001F86188A60C02434310529F02335310548
:102CF00009F4B2C092C064E482EE95E00E94782AA2
:102D00002AE030E040E054E76BE872E382EE95E0C1
:102D10000E94062B6CE282EE95E00E94782A2AE05F
:102D200030E040E05EEC6DEE74E382EE95E00E94F0
:102D3000062B6CE282EE95E00E94B82AADCF0F5FC1
:102D4000043009F0A9CF29813A814B815C81A8EE3A
:102D5000B3E00E94DB2D698B7A8B8B8B9C8B2D8152
:102D60003E814F8158850E94DB2D698F7A8F8B8F32
:102D70009C8F29853A854B855C852D8F3E8F4F8FA3
:102D800058A32D853E854F8558890E94DB2D6B0108
:102D90007C0160323EE473078105910530F462E303
:102DA0008CE10E94D10900E077CF603345E77407DA
:102DB0008105910510F462E2F3CF60345CE9750798
:102DC0008105910510F466E2EBCF80E5C81683EC2F
:102DD000D806E104F10410F462E1E2CF90E6C916EE
:102DE0009AEED906E104F10410F465E1D9CFA0E729
:102DF000CA16A1E1DA06A1E0EA06F10410F461E0E6
:102E0000CFCFB0EACB16B6E8DB06B1E0EB06F104B3
:102E100010F463E0C5CF65E0C3CF10ED180F1A3092
:102E200008F03ACFE1E0F0E0EC0FFD1F24E0029F54
:102E3000E00DF11D11242081318142815381AAE0EE
:102E4000B0E00E94DB2D610F711D811D911D60831B
:102E500071838283938320CF49885A886B887C88CA
:102E6000812C912C540118CF81149104A104B10438
:102E700089F4C301B2010E94400A61E070E080E081
:102E800090E00E94DD281D8A1E8A1F8A188E312C30
:102E900022242A948D8D9E8DAF8DB8A18816990617
:102EA000AA06BB06D0F40E94FA092D893E894F89F3
:102EB000588D280F311D411D511D2D8B3E8B4F8B81
:102EC000588F381608F4382E821508F4282E3FEF54
:102ED000831A930AA30AB30A56C0C301B20128EEAB
:102EE00033E040E050E00E94122EBA01A9012AE02E
:102EF00030E082EE95E00E945D2B6CE282EE95E080
:102F00000E94782A4AE050E0632D82EE95E00E940C
:102F10006C2B6CE282EE95E00E94782A6D897E89A6
:102F20008F89988DA50194010E94122EBA01A901E2
:102F30002AE030E082EE95E00E945D2B6CE282EEAA
:102F400095E00E94782A4AE050E0622D82EE95E0FA
:102F50000E946C2B6CE282EE95E00E94B82A4C0C29
:102F60005D1C6E1C7F1C898D9A8DAB8DBC8D84156C
:102F70009505A605B70520F449885A886B887C8892
:102F8000812C912C540129893A894B895C89283EEE
:102F900033404105510509F07FCEA296E2E10C9441
:102FA0006F2EACE1B0E0E7EDF7E10C945D2E0E94EE
:102FB000BA286B017C0181E00E94B00A14E703E0AB
:102FC000198361E0CE0101960E940D0C00937305F8
:102FD0000E948B0B6AEF70E080E090E00E94DD2899
:102FE00080917305833089F482EE95E00E94BA2BBC
:102FF000892B59F40E94BA286C197D098E099F0902
:103000006038734C894C9140D8F2809173058330BD
:1030100009F44FC08FE70E94A9090E94BC09898367
:10302000843511F083E05CC00E94BC091092460513
:10303000809347050E94BC092091460530914705C1
:10304000280F311D30934705209346050E94BC0987
:10305000809348050E94BC0980934905813110F78F
:10306000F12C0F2D10E08091490590E0880F991FF9
:103070000817190740F40E94BC09F801E65BFA4FF3
:103080008083F394EECF80E7898361E0CE010196DF
:103090000E940D0C83E0809373050E948B0B62E30A
:1030A00070E080E090E00E94DD288091730583301D
:1030B00011F482E015C08FE70E94A9090E94BC09A3
:1030C0008983803509F0AECF0FE915E00E94BC0975
:1030D000F80181938F01F5E00A3B1F07B9F781E002
:1030E0006C96E8E00C94792E80914505992787FD30
:1030F0009095A92FB92FFC013196EB30F10508F01E
:1031000066C0EC5CFF4F0C948A2E62E778E082EE9A
:1031100095E00E94942A82E893E00E94620C6AE59E
:1031200078E082EE95E00E94942A65E378E082EEF2
:1031300095E00E94942A6BE078E082EE95E00E9490
:10314000942A6AEE77E082EE95E00E94942A6DEB75
:1031500077E082EE95E00E94942A67E977E082EEBC
:1031600095E00E94942A63E777E082EE95E00E9462
:10317000942A6CE477E082EE95E00E94942A82EE35
:1031800095E00E94802A0E94A20D21C06FE277E0A4
:103190001AC06AE077E017C065EF76E014C066ED0C
:1031A00076E011C062E976E00EC06DE776E00BC014
:1031B00068E676E082EE95E00E94942A62E276E08C
:1031C00002C06CE076E082EE95E00E94942A6AE00C
:1031D00070E080E090E00E94DD2882EE95E00E94A1
:1031E000BA2B892B29F082EE95E00E94E72BF5CFD0
:1031F0000895ACE1B0E0EFEFF8E10C945D2E909112
:1032000045059F3F09F023C1482F50E0FA013A9746
:10321000EF36F10508F00FC1E15CFF4F0C948A2EE8
:1032200061E172E0A0C06DE172E082EE95E00E9483
:10323000A62A85E789838BE1EFE9F5E0DE011296A6
:1032400001900D928A95E1F76CE1CE0101960E9402
:103250000D0C0E948B0B83E08093730568EC70E08B
:1032600080E090E00E94DD2880917305843009F0B1
:10327000E2C08FE70E94A9090E94BC0989838535B5
:1032800009F0D9C06DEE74E082EE95E00E94942AB8
:103290006FEC74E082EE95E00E94942A61EB74E09A
:1032A00096C065E372E082EE95E00E94A62A89E668
:1032B000898361E0CE0101960E940D0C0E948B0B68
:1032C00083E08093730568EC70E080E090E00E94FA
:1032D000DD2880917305843009F0ADC08FE70E942E
:1032E000A9090E94BC0989838E010E5F1F4F7E01D0
:1032F0004DE1E40EF11C0E94BC09F80181938F019D
:10330000EE15FF05C1F78BE1FE013296AFE9B5E09E
:1033100001900D928A95E1F78981893409F08BC07B
:1033200063E974E082EE95E00E94942A65E774E018
:1033300082EE95E00E94942A67E574E048C06FE44D
:1033400072E082EE95E00E94A62A8EEF80934505FA
:1033500072C080528750805390914805981708F0AA
:1033600066C06EE572E082EE95E00E94A62A63C018
:1033700084E18093450560E274E029C085E1809393
:10338000450569EE73E023C086E18093450562EB55
:1033900073E01DC087E18093450568E673E017C0C0
:1033A00088E18093450567E573E011C089E180936A
:1033B000450563E473E00BC08AE1809345056EE246
:1033C00073E005C08BE18093450566E073E082EE13
:1033D00095E00E94942A2FC06CEE72E082EE95E098
:1033E0000E94942A8091AD0591E01DC066ED72E0C7
:1033F00082EE95E00E94942A8091AD0592E013C080
:1034000061EC72E082EE95E00E94942A8091AD0515
:1034100094E009C066EA72E082EE95E00E94942A88
:103420008091AD0598E089278093AD058FEF80935B
:1034300045050E94431082EE95E00E94BA2B892B2D
:1034400009F45AC182EE95E00E94E72BF4CF0E9466
:103450004211882309F450C18091DF04811104C016
:103460008FEF8093450540C140E050E060E070E0A0
:1034700080EE94E00E94012F40914505042F112712
:1034800007FD1095212F312FF8013197EB31F10510
:1034900008F01AC1E255FF4F0C948A2E552747FDBC
:1034A00050952091480530E0241735070CF40CC1E5
:1034B0008B019C01015011092109310900321105CC
:1034C0002105310558F0C0904905EBE4F5E0F12CF9
:1034D000D12CA8E2EA2E415051090FC0FA01E15661
:1034E000FA4F61506083D8C0DF0111972C9130E012
:1034F0002417350729F0F3943296FC10F5CFCAC093
:103500000E2D10E020E030E00617170728073907D6
:1035100041F42081DA01A156BA4F11962C93DD2493
:10352000D394E394E8CF6F3F71058105910511F0C5
:1035300008F0CAC06093B705AFC06F3F7105810541
:10354000910511F008F0C0C06093B805A5C06F3FA9
:1035500071058105910511F008F0B6C06093B905B9
:103560009BC02091E00420622037E9F440E050E065
:1035700060E070E081EE94E00E94012F9B01AC01BD
:10358000DC01CB010197A109B1090897A105B1059B
:1035900008F0ADC0A4EDB0E30E94DB2D6A5E7C4A6A
:1035A0008A46954E24C02636E9F440E050E060E0BB
:1035B00070E081EE94E00E94012F9B01AC01DC01E0
:1035C000CB010197A109B1090797A105B10508F041
:1035D0008EC0A8EAB1E60E94DB2D645E7C438E4675
:1035E000944E05C0611571058105910571F08B013F
:1035F0009C0114572B4832430130FAE51F07F2E6CD
:103600002F07F2E03F0708F05FC06093AF057093AB
:10361000B0058093B1059093B2053EC06F3F710530
:103620008105910511F008F04FC06093B30534C0D7
:103630008B019C0101501109210931090F3F11052E
:103640002105310508F040C06093B40525C08B0109
:103650009C01045C1940210931090D344DE1140726
:103660002105310528F47093B6056093B50514C0A3
:10367000611571058105910521F48FEF8093AE05E9
:103680000BC06134710581059105F0F461506093C0
:10369000AE0502C0DD20C1F08091DE0481111AC0A8
:1036A00080917F0590918005A0918105B091820560
:1036B0000196A11DB11D80937F0590938005A09375
:1036C0008105B093820506C060E772E082EE95E066
:1036D0000E94A62A0E9438118FEF809345056AE068
:1036E00082EE95E00E94B82A0E94431005C061E076
:1036F00070E080E090E07BCF6C96E8E00C94792E4F
:103700006AE572E082EE95E00E94942A62E472E03B
:1037100082EE95E00E94942A82EE95E00E94BA2BF8
:10372000892B31F082EE95E00E94E72B0E94F91878
:103730000E94D117823029F0833051F46DE072E09D
:1037400002C064E272E082EE95E00E94942A08953D
:103750008FEF809345051092DE040E944310809104
:1037600045058E3F69F082EE95E00E94BA2B892BC9
:10377000B1F382EE95E00E94E72B0E94F918EFCF9B
:1037800008950F931F93109145051F3F09F0D2C074
:10379000893409F457C000F5883309F469C058F436
:1037A000803309F477C008F061C08B3109F440C060
:1037B0008132B1F1B9C0813409F487C030F4893362
:1037C00009F466C0803461F1AFC0823409F48EC060
:1037D000863409F448C0A8C0823609F487C078F45A
:1037E000883531F128F48235C1F18335E1F09CC090
:1037F0008A3509F494C0813609F467C095C08237D0
:1038000061F128F4863679F18936E1F08DC0883788
:1038100079F08A3709F483C0833709F085C003C083
:1038200061E172E015C00E94730D6EE872E004C0A1
:103830000E947C0D68EA72E082EE95E00E94A62A62
:103840008EEF70C00E947A060E94BF0667EC72E09D
:1038500082EE95E00E94A62A67C081E00E94DF0602
:1038600060EE72E0F5CF0E94ED105EC080535AC04A
:103870006AEF71E082EE95E00E94942A90919E0595
:1038800088E0890F8871977E892B80939E051AC0E6
:1038900089E048C067EE71E082EE95E00E94942ACC
:1038A0008091BF059091C005A091C105B091C2055E
:1038B00020E182278093BF059093C005A093C105A6
:1038C000B093C205109345052FC061ED71E082EE03
:1038D00095E00E94942A8091BF059091C005A09127
:1038E000C105B091C20540E4842710C060EC71E0CE
:1038F00082EE95E00E94942A8091BF059091C005C8
:10390000A091C105B091C20520E282278093BF0536
:103910009093C005A093C105B093C20502C00E9458
:10392000801B8FEF80934505809145058E3F09F000
:10393000D4C0DDC00E944211882309F4D8C0809110
:10394000DF04811104C08FEF80934505C6C040E0BD
:1039500050E060E070E080EE94E00E94012F009162
:103960004505112707FD1095212F312FF8013197BB
:10397000E930F10508F0B4C0E753FF4F0C948A2EEC
:103980008B019C01015014472B4832430F3F1945CE
:103990002246324008F0A4C060937B0570937C05FA
:1039A00080937D0590937E0577C060937F0570932B
:1039B0008005809381059093820581E08093DE04E9
:1039C0006BC0683071058105910508F089C060936E
:1039D000830562C08B019C01015011092109310945
:1039E0000A3011052105310508F07AC0609384057D
:1039F00053C061EB71E080EE94E00E943B3010E038
:103A0000009799F00E941530009779F0183130F442
:103A1000E12FF0E0EA58FA4F87871F5F61EB71E012
:103A200080E090E00E943B30EBCF1831A8F5E12F09
:103A3000F0E0EA58FA4F17861F5FF7CF653071053F
:103A40008105910508F04CC060939D0525C08B0150
:103A50009C01015011092109310906301105210588
:103A60003105F0F520919E05287F262B20939E0599
:103A700013C08B019C010150110921093109011565
:103A8000124C2140310560F56093770570937805FD
:103A90008093790590937A058091DE04811113C09B
:103AA00080917F0590918005A0918105B09182055C
:103AB0000196A11DB11D80937F0590938005A09371
:103AC0008105B09382050E9438118FEF80934505E0
:103AD0006AE082EE95E00E94B82A0E94741807C03E
:103AE00060E772E082EE95E00E94A62AECCF1F917B
:103AF0000F9108958FEF809345051092DE040E9488
:103B00007418809145058E3F69F082EE95E00E9421
:103B1000BA2B892BB1F382EE95E00E94E72B0E942D
:103B2000C11BEFCF6AE070E080E090E00E94DD28EA
:103B300082EE95E00E94BA2B892B29F082EE95E067
:103B40000E94E72BF5CF0895CF93C82F682F82EE00
:103B500095E00E94142C90916A059C2790936A0529
:103B6000CF910895A1E0B0E0E8EBFDE10C94632E65
:103B700099830E94A41D9981892F0E94A41D2196DA
:103B8000E2E00C947F2E1F93CF93DF93182FEB016D
:103B900010926A0565EB70E082EE95E00E9459068E
:103BA00062E670E082EE95E00E945906812F0E9445
:103BB000A41DCE010E94B21DDF91CF911F910895E7
:103BC00060916A0582EE95E00E94142C0895A1E2AE
:103BD000B0E0EDEEFDE10C945F2E7B018A018C30AC
:103BE00009F453C108F040C0863009F4BCC018F590
:103BF000833009F491C070F4813009F472C08230CE
:103C000009F048C26BE170E082E00E94C31D0FE939
:103C100015E078C0843009F487C0853009F03AC2D5
:103C20006091490570E0660F771F85E00E94C31D13
:103C30000AE415E086C0893009F4A7C070F4873023
:103C400009F49BC0883009F025C261E070E088E08B
:103C50000E94C31D8091D40523C28A3009F4CAC0D2
:103C60008B3009F4F2C016C28A3609F475C1D8F453
:103C7000873609F43AC138F4853609F40EC1863620
:103C800009F41FC107C2883609F437C1893609F023
:103C900001C261E070E089E60E94C31D0E947A06BD
:103CA0000E94BF06F5C18D3609F4D4C138F48B36B5
:103CB00009F491C18C3609F49AC1ECC18E3609F42D
:103CC000DCC1873C09F0E6C161E070E087EC0E944E
:103CD000C31D81E00E94A41D0E94E01D10926B058F
:103CE000E3C169E270E081E00E94C31D06E715E0D0
:103CF000F80181918F010E94A41DF5E00F391F0783
:103D0000B9F7D0C1F80181918F010E94A41DF5E09F
:103D10000A3B1F07B9F7C6C161E070E083E00E946B
:103D2000C31D0E94D117BCC161E070E084E00E9415
:103D3000C31D81E00E94A41D0E94E01D0E94051683
:103D4000B3C18091490590E0880F991F98012A54CA
:103D500035402817390708F0A5C1F80181918F0176
:103D60000E94A41DEECF62E070E086E00E94C31DB9
:103D700082E893E00E94B21D95C161E070E087E0A7
:103D80000E94C31D809148058BC186E6898361E04E
:103D9000CE0101960E940D0C0E948B0B83E0809354
:103DA000730568EC70E080E090E00E94DD2880916F
:103DB00073058430D9F48FE70E94A9090E94BC09D9
:103DC0008983863469F460E270E089E00E94C31D53
:103DD00010E20E94BC090E94A41D1150D1F762C1DB
:103DE00061E070E089E00E94C31D52C161E070E0B3
:103DF00089E053C169E170E08AE00E94C31D81E05F
:103E00008093BA05209172058091BF059091C005FD
:103E1000A091C105B091C205222311F0806801C0B4
:103E20008F778093BF059093C005A093C105B09391
:103E3000C2050AEB15E0F80181918F010E94A41DD3
:103E4000F5E0033D1F07B9F72DC161E270E08BE09B
:103E50000E94C31D8091AA048F3F39F08091AA046B
:103E600091E0980F9093AA0402C08091AA040E9446
:103E7000A41D10E0812F0E94E7150E943C090E94BA
:103E8000B21D1F5F1031B1F70DC161E070E08CE031
:103E90000E94C31D8091D30503C161E070E085E6F7
:103EA0000E94C31D89E2E816F10409F0F8C0D801A8
:103EB000E6E7F5E08D91819385E0EF39F807D1F7DA
:103EC000E7C061E070E086E60E94C31DEBE1EE16FC
:103ED000F10409F0E4C0D801EFE9F5E08D91819398
:103EE00085E0EA3BF807D1F7D3C061E070E087E6F0
:103EF0000E94C31D0E94730DCBC061E070E088E694
:103F00000E94C31D85E789838BE1EFE9F5E0DE01BF
:103F1000129601900D928A95E1F76CE1CE0101961F
:103F20000E940D0C0E948B0B83E08093730560E26E
:103F300073E080E090E00E94DD288091730584307A
:103F400009F0ADC08FE70E94A9090E94BC098983CE
:103F5000853509F0A4C09CC061E070E08AE60E944B
:103F6000C31D89E6898361E0CE0101960E940D0C94
:103F70000E948B0B83E08093730560E273E080E026
:103F800090E00E94DD2880917305843009F087C09D
:103F90008FE70E94A9090E94BC0989838E010E5FE8
:103FA0001F4F7E01EDE1EE0EF11C0E94BC09F801ED
:103FB00081938F01EE15FF05C1F78BE1FE0132966B
:103FC000AFE9B5E001900D928A95E1F789818934D6
:103FD00009F065C05DC061E070E08BE60E94C31D22
:103FE000F80180818093D4050E947C0D51C061E06E
:103FF00070E08CE60E94C31DF0E2EF16F10461F45C
:1040000087E6898380E2F801DE01129601900D9225
:104010008A95E1F761E203C087E4898361E0CE011C
:1040200001960E940D0C0E948B0B83E08093730518
:104030006CE474E080E090E00E94DD2880917305DC
:10404000843069F58FE70E94A9090E94BC09873472
:1040500031F51EC061E070E08DE60E94C31D89E16C
:10406000E816F104E1F4D801EAEBF5E08D918193D3
:1040700085E0E33DF807D1F70BC061E070E08EE624
:104080000E94C31DF80180818093D3050E945D0DBD
:1040900081E006C061E070E08AEC0E94C31D80E010
:1040A0000E94A41D0E94E01DA196E6E00C947B2EC8
:1040B000A0E0B0E0EEE5F0E20C945D2ECAECD3E0B7
:1040C00014E606E035E0F32E44E0E42E53E0D52E6E
:1040D00062E0C62E82EE95E00E94BA2B892B09F48D
:1040E0009BC082EE95E00E94E72B282F8093350439
:1040F0004091340450E04730510560F7FA01EE5228
:10410000FF4F0C948A2E853B29F781E0809334047D
:10411000E1CF823609F07DC0C0923404DBCF8093BA
:10412000330480933204D0923404D4CF9C013327DB
:104130003093310420933004909132049827909367
:104140003204E0923404C6CF382F22274091300445
:1041500050913104242B352B3093310420933004BB
:1041600090913204982790933204F09234042536CB
:10417000310508F4AFCF61E070E08CEC0E94C31D04
:1041800081E00E94A41D0E94E01D43C020912E04E6
:1041900030912F04F901E653FC4F80839091320453
:1041A000982790933204C901019690932F0480932D
:1041B0002E0420913004309131048217930708F4C3
:1041C00089CF0093340486CF8091320482130BC0D0
:1041D00060912E0470912F044AEC53E080913304D7
:1041E0000E94E71D0DC062E070E08BEC0E94C31DD1
:1041F000809133040E94A41D80916A050E94A41D31
:10420000FE01812F11928A95E9F710922F041092E6
:104210002E04109234045ECFCDB7DEB7E8E00C94E4
:10422000792E81E080936B0580916B05882349F09E
:1042300082EE95E00E94BA2B892BB1F30E945820A0
:10424000F3CF0895AAE2B0E0E8E2F1E20C945B2E2D
:104250000E94AE286B017C0181E00E94B00A82EED0
:1042600095E00E94BA2B892B29F082EE95E00E94FE
:10427000E72BF5CF4398299811E072E6B72EE9E2D3
:10428000AE2E03E00E94AE286C197D098E099F09AD
:10429000693C710581059105F0F11123E1F10E945E
:1042A000AE286B017C0185B1846285B980ED97E011
:1042B0000E94B607B982E6E7F5E0DE0112968A2D84
:1042C00001900D928A95E1F76AE2CE0101960E9473
:1042D0000D0C85B18B7D85B980E090E00E94B6071A
:1042E000009373050E948B0B62E370E080E090E026
:1042F0000E94DD2880917305843061F4009373057A
:104300008FE70E94A9090E94BC0911E0823419F4C8
:1043100010E001C011E087E00E94D329892BB1F49D
:1043200011E014C0439A299A85B1846285B982EE5E
:1043300095E00E94E72B8D309105C1F074F40A9747
:10434000A9F04398299885B18B7D85B982EE95E0D7
:104350000E94BA2B892B31F795CF8332910579F0E2
:104360008234910571F70E941121EBCF62EB71E06D
:1043700082EE95E00E94942A0E947A1DE2CF0E946C
:104380000516DFCF8F929F92AF92BF92CF92DF92AE
:10439000EF92FF921F93CF93DF9387E00E94D32980
:1043A000892B09F089C068EC70E080E090E00E9401
:1043B000DD2880E090E00E94B6070E94AE284B0105
:1043C0005C016B017C0180ECC80E82E1D81EE11C0F
:1043D000F11C0E94AE286C157D058E059F0530F4FA
:1043E00087E00E94D329892BA1F364C087E00E9453
:1043F000D329892B09F05EC080ED97E00E94B607B3
:104400000E94AE286B017C01D0E0C1E088E4880EF8
:1044100086E2981EA11CB11C11E087E00E94D329FE
:10442000892B21F58C149D04AE04BF0430F480ED7B
:1044300097E00E94B607D1E0F0CF0E94AE286C1939
:104440007D098E099F09693C71058105910528F355
:104450000E94AE286B017C01C12719F080ED97E026
:1044600002C080E090E00E94B607D7CF80E090E0E5
:104470000E94B607DD23B9F08091D30590E0019644
:1044800065E070E00E94FE2D8093D3050E945D0DD3
:104490000E94DC130E947C0D64EF71E080E090E0EC
:1044A0000E94DD2809C080E00E94DF060E94F4110E
:1044B0000E94730D0E942221DF91CF911F91FF90E6
:1044C000EF90DF90CF90BF90AF909F908F90089526
:1044D000CF92DF92EF92FF9280E00E940D080E943F
:1044E000E40761E081E10E94672961E08DE00E94BC
:1044F000672961E089E00E94672961E08AE00E9403
:10450000672960E087E00E94672960E088E00E94F8
:10451000672961E088E00E94A0290E949F0740E08F
:1045200052EC61E070E082EE95E00E94022D0E9464
:10453000DC130E947C0D0E94C1138FEF8093AA04AC
:104540000E94F90778940E94AE286B017C0180914B
:10455000AA048F3F59F40E94AE286C197D098E0978
:104560009F09603D77408105910588F380ED97E0D4
:104570000E94B60761E087E00E94A029439A299A29
:1045800082EE95E00E94BA2B892B29F082EE95E00D
:104590000E94E72BF5CF6DEF72E082EE95E00E946E
:1045A000752A82E893E00E94620C64E173E082EE77
:1045B00095E00E94752A4AE050E063E070E082EEE8
:1045C00095E00E94452B62E370E080E090E00E945D
:1045D000DD2882EE95E00E94BA2B04970CF182EE62
:1045E00095E00E94E72B82349105D1F482EE95E0AC
:1045F0000E94E72B8E34910599F482EE95E00E949B
:10460000E72B8434910561F482EE95E00E94E72B5C
:10461000819731F480E090E00E94B6070E94222149
:1046200040917705509178056091790570917A05F0
:10463000DB01CA010197A109B1090497A105B105E0
:1046400068F44093A904433029F440EA56E861E055
:1046500070E004C040E052EC61E070E082EE95E072
:104660000E94022D0E94C2214398299880E090E088
:104670000E94B6070E94C1131092C5048091BF0525
:1046800083FF11C080918B05882351F080919205A2
:10469000882331F080919905882311F087E001C0CB
:1046A00085E08093C50480E00E94B00A8091C60432
:1046B0000E94E4090E948B0B10923F0410923E046A
:1046C00010923D04F12C8091D4058F15B0F062E377
:1046D00070E080E090E00E94DD2880ED97E00E948D
:1046E000B60762E370E080E090E00E94DD2880E0A1
:1046F00090E00E94B607F394E6CF80919E0584FF78
:1047000008C0982F987181E0983109F080E00E94EC
:10471000B0118FE00E940D08FF90EF90DF90CF90D6
:104720000895EF92FF920F931F93CF93DF938C0125
:104730006EE770E082EE95E00E945906E801F12CE8
:10474000F0E2EF2E8E0188818D57823048F46DE7BC
:1047500070E082EE95E00E94590688818E2588835C
:104760002196F801608182EE95E00E94142CF3946A
:10477000F9E0FF12E7CF6EE770E082EE95E00E946D
:104780005906CDB7DEB7E6E00C947B2EA9E0B0E089
:10479000ECECF3E20C94632E9091C70491110EC0DF
:1047A0009EEF99838A836B8350E0559547954C83A0
:1047B0002D83198618861F821E822EC04091CC043C
:1047C000842F90E0B4E095958795BA95E1F7242F72
:1047D0002F7030E08217930719F18DEF89831B82C8
:1047E000FE01349650E0842F90E0A4E095958795E3
:1047F000AA95E1F7242F2F7030E08217930749F034
:10480000DC01A353BB4F8C918193405F5F5F5630B7
:1048100051F74093CC045A83CE0101960E94912314
:104820008091C70490E0019666E070E00E94FE2D42
:104830008093C7042996E2E00C947F2EA0E0B0E0BC
:10484000E4E2F4E20C945C2E6C016EE770E082EE20
:1048500095E00E9459068601E12CF12CC0E0D0E0E1
:1048600030E2B32EF801608183E8860F823078F45D
:104870006DE770E082EE95E00E945906F8016081D4
:104880006B2570E082EE95E00E94590604C082EE2E
:1048900095E00E94142CE114F10459F0F801808194
:1048A0009E01280F311DC901C92FDD27C80FD91F4F
:1048B000DD273FEFE31AF30A89E0E816F10459F027
:1048C00028E0E216F10421F48C2F8095F601808710
:1048D0000F5F1F4FC7CFCDB7DEB7E9E00C94782E3E
:1048E000A9E0B0E0E6E7F4E20C94632EE82F362F5F
:1048F0008091C70490E0019664E270E00E94FE2D72
:104900008093C70458E9598350E15A83813089F074
:1049100048F08230B9F08330D9F48B8381EF8C83F7
:104920003D8319C085E08B8381EF8C832F5F2D83BE
:1049300012C08B8381EF8C8384E6489FA0011124F1
:104940005D8309C084E08B8381EF8C83ED8303C09A
:104950000E94ED1104C0CE0101960E941E242996EA
:10496000E2E00C947F2EA2E0B0E0E9EBF4E20C94DC
:10497000582E182F762E2A8349830E94BA286B015D
:104980007C018091DD048090C8049090C904A090BF
:10499000CA04B090CB042A8149818823C1F0D70191
:1049A000C60188199909AA09BB094C015D0191EE5C
:1049B00089169EE29906A104B10420F1241708F497
:1049C000422F202F672D812F0E94702413C0D70102
:1049D000C60188199909AA09BB094C015D0191E337
:1049E000891695E79906A104B10460F0672D812F1F
:1049F0000E94C623C092C804D092C904E092CA049F
:104A0000F092CB042296EDE00C94742EA2E2B0E07A
:104A1000ECE0F5E20C94592E8CE00E94CB09811158
:104A20000FC06CE173E082EE95E00E94A62A439AE3
:104A3000299A80E00E94B00A0E948B0B4398299823
:104A400082EE95E00E94BA2B892B01F182EE95E06F
:104A50000E94E72B9091A904992319F00E94EF136B
:104A6000EFCF40913E0450E09A012F5F3F4F2F71EE
:104A7000332760913F0470E02617370709F3FA01E6
:104A8000E75BFB4F808320933E04DACF8091730570
:104A9000843009F086C00E94BA286115710581052D
:104AA000910549F06093B7047093B8048093B904FA
:104AB0009093BA040CC081E090E0A0E0B0E0809355
:104AC000B7049093B804A093B904B093BA0480914A
:104AD000AD049091AE0481609093AE048093AD04D8
:104AE00083E0809373058FE70E94A90909E614E02B
:104AF0000E94BC09F80181938F01F4E002371F077F
:104B0000B9F72091720480916904982F922796FF3B
:104B10003BC090E4922790937204982F9873983337
:104B2000F1F410E0212F30E080916904877090E06B
:104B3000821793074CF11F5F20919E05812F90E013
:104B4000FC01E759FB4F24FF04C080810E94CF1174
:104B5000E9CF608182EE95E00E94142CE3CF8F7341
:104B600099F480916A048093B60480916B048093D9
:104B7000B40480916C048093B30480916F0490E03E
:104B80009093AC048093AB0480913D04813019F480
:104B900082E080933D0480913D04833011F41092B3
:104BA0003D040E94BA286B017C018091AF04909172
:104BB000B004A091B104B091B2040097A105B10571
:104BC000C9F0A7019601281B390B4A0B5B0BDA01D0
:104BD000C901883B9B40A105B10560F00E94FA091C
:104BE0008093B5041092AF041092B0041092B104F7
:104BF0001092B2048091BB049091BC04A091BD04BA
:104C0000B091BE0446015701881A990AAA0ABB0A44
:104C100086E795E00E94270886169706A806B9063B
:104C200008F4AAC0C092BB04D092BC04E092BD04B8
:104C3000F092BE040E9457068091AA048830A0F02A
:104C40008091BF059091C005A091C105B091C205AA
:104C50005CE1B695A795979587955A95D1F7892BDD
:104C60008A2B8B2B09F0A4C18091AA048F5F8093BB
:104C7000AA048091B7049091B804A091B904B091AE
:104C8000BA040097A105B105F1F0C81AD90AEA0AD9
:104C9000FB0A86E795E00E9427086C157D058E05C6
:104CA0009F0508F00AC18091BF0584FD04C080ED16
:104CB00097E00E94B6071092B7041092B8041092C1
:104CC000B9041092BA0490917204907C909372048B
:104CD00050913E0480913F0420913D04581709F4FF
:104CE00009C1223009F006C1905890937204E091F6
:104CF0009E05E770F0E0E658FC4F6081693008F0EF
:104D0000E1C0615040E04613DFC080933F0487E379
:104D1000840F90917204892B809372044093400415
:104D200083E080933D0485B1846285B980918305D9
:104D30009091C50491112DC10E94AB0A8091C604C7
:104D40000E94E409E0919E05E770F0E0E658FC4F10
:104D5000608182E794E00E94C60BE091C604EF5F99
:104D6000E093C604E83109F420C1F0E0EA58FA4FB4
:104D70008785882309F419C10E94350C813069F5B3
:104D800080919E05887149F18091AD049091AE04A7
:104D9000880F991F9093AE048093AD0483E08093B5
:104DA00073050E948B0B0E94BA286093AF04709326
:104DB000B0048093B1049093B204672B682B692BE5
:104DC00061F481E090E0A0E0B0E08093AF049093C4
:104DD000B004A093B104B093B20480919E0584FF07
:104DE0001FC08091AD049091AE048E7F0E945D093A
:104DF000182F6091AB048091B6040E94E513482FF0
:104E0000612F8091B50449A30E94E5130091D40558
:104E1000282F49A16091B3048091B4040E94B32467
:104E200085B18B7D85B98091C3048130C1F018F0C4
:104E30008230B1F1CBC087E00E94D329892B09F0E1
:104E4000C5C081E08093C3040E94AE286093BF0474
:104E50007093C0048093C1049093C204B7C087E0EC
:104E60000E94D329892B31F50E94AE28C090BF043F
:104E7000D090C004E090C104F090C2046C197D0988
:104E80008E099F09693E73408105910508F49EC013
:104E900082E08093C30480ED97E00E94B60796C03D
:104EA00087E00E94D329892B09F490C080E090E02C
:104EB0000E94B6071092C30489C080E090E00E946F
:104EC000B60701CF68E01ECF851709F41ECF4F5FEC
:104ED000242F30E090E0F901EE58FB4FDC01A75B96
:104EE000BB4F7C917083F901E05CFB4F70830196AE
:104EF0008F7109CF2430B1F42091400481E494E013
:104F0000A3E7B4E0FC013E2F381B321718F43191AF
:104F10003D93F9CF87E3820F90917204892B8093A0
:104F20007204FECE8091C304823059F49160909354
:104F30007204439A299A8E010F5F1F4FF12CB8011A
:104F400011C04398299880913D04811103C081E0EC
:104F500080933D0480913D04833069F784E0809321
:104F60003D04E9CF8F2D69A37AA30E94E715F801CC
:104F7000819391938F01F39469A17AA1F0E1FF12DB
:104F8000F1CF80919E0543E754E087700E94AC0802
:104F9000CACE882309F4D0CE2091C40431E0320F68
:104FA0003093C4042913C8CE0DC01092C604E4CEB9
:104FB0008091AA04883011F4439A299A89E0809359
:104FC000AA04DACE1092C4048150B6CEA296ECE0C8
:104FD0000C94752E8230E8F4E82FF0E0EE0FFF1FFE
:104FE000EB52FA4F71836083813041F08091690008
:104FF0008C7F842B80936900E89A089580916900E2
:10500000440F551F440F551F837F842B80936900E5
:10501000E99A08951F920F920FB60F9211242F93C1
:105020003F934F935F936F937F938F939F93AF9330
:10503000BF93EF93FF938091D5059091D605892B6F
:1050400029F0E091D505F091D6050995FF91EF91F2
:10505000BF91AF919F918F917F916F915F914F9190
:105060003F912F910F900FBE0F901F9018951F9298
:105070000F920FB60F9211242F933F934F935F938C
:105080006F937F938F939F93AF93BF93EF93FF9310
:105090008091D7059091D805892B29F0E091D7050B
:1050A000F091D8050995FF91EF91BF91AF919F9134
:1050B0008F917F916F915F914F913F912F910F90C1
:1050C0000FBE0F901F9018951F920F920FB60F9260
:1050D00011242F933F938F939F93AF93BF9380910E
:1050E000DA059091DB05A091DC05B091DD053091EA
:1050F000D90523E0230F2D3720F40196A11DB11D02
:1051000005C026E8230F0296A11DB11D2093D905E5
:105110008093DA059093DB05A093DC05B093DD0561
:105120008091DE059091DF05A091E005B091E10549
:105130000196A11DB11D8093DE059093DF05A0931C
:10514000E005B093E105BF91AF919F918F913F91A1
:105150002F910F900FBE0F901F9018952FB7F894B6
:105160006091DA057091DB058091DC059091DD0599
:105170002FBF08953FB7F8948091DE059091DF0529
:10518000A091E005B091E10526B5A89B05C02F3F91
:1051900019F00196A11DB11D3FBF6627782F892FF9
:1051A0009A2F620F711D811D911D42E0660F771FBE
:1051B000881F991F4A95D1F70895CF92DF92EF92F9
:1051C000FF92CF93DF936B017C010E94BA28EB0121
:1051D000C114D104E104F10479F00E94BA286C1BD7
:1051E0007D0B683E7340A0F381E0C81AD108E10846
:1051F000F108C851DC4FECCFDF91CF91FF90EF90D9
:10520000DF90CF900895789484B5826084BD84B592
:10521000816084BD85B5826085BD85B5816085BDB1
:10522000EEE6F0E0808181608083E1E8F0E01082CA
:10523000808182608083808181608083E0E8F0E00B
:10524000808181608083E1EBF0E0808184608083F5
:10525000E0EBF0E0808181608083EAE7F0E080812C
:10526000846080838081826080838081816080838C
:105270008081806880831092C1000895833081F01E
:1052800028F4813099F08230A1F008958630A9F099
:105290008730B9F08430D1F4809180008F7D03C0D5
:1052A000809180008F7780938000089584B58F77F8
:1052B00002C084B58F7D84BD08958091B0008F7742
:1052C00003C08091B0008F7D8093B0000895CF938C
:1052D000DF9390E0FC01ED50F44F2491FC01E95F75
:1052E000F34F8491882349F190E0880F991FFC01C6
:1052F000E15DF34FA591B4918B5D934FFC01C59196
:10530000D4919FB7611108C0F8948C9120958223A5
:105310008C93888182230AC0623051F4F8948C9176
:10532000322F309583238C938881822B888304C00D
:10533000F8948C91822B8C939FBFDF91CF9108952D
:10534000A1E0B0E0E6EAF9E20C94612E282F30E00B
:10535000F901E152F44F8491F901ED50F44F1491A9
:10536000F901E95FF34F04910023C9F0882321F08C
:1053700069830E943E296981E02FF0E0EE0FFF1F54
:10538000EB5DF34FA591B4919FB7F8948C916111A7
:1053900003C01095812301C0812B8C939FBF219660
:1053A000E4E00C947D2ECF93DF93282F30E0F901B9
:1053B000E152F44F8491F901ED50F44FD491F90189
:1053C000E95FF34FC491CC2391F081110E943E29F3
:1053D000EC2FF0E0EE0FFF1FE55EF34FA591B491C7
:1053E0002C912D2381E090E021F480E002C080E048
:1053F00090E0DF91CF9108958E3008F08E50877045
:1054000020919D0190E4299F90011124822B80938B
:105410007C0080917A00806480937A0080917A0089
:1054200086FDFCCF809178002091790090E0922B4E
:105430000895A0E0B0E0EFE1FAE20C945D2E6C017B
:105440007A01EB01E60EF71E00E010E0CE15DF0555
:1054500061F06991D601ED91FC910190F081E02D10
:10546000C6010995080F191FF1CFC801CDB7DEB7E6
:10547000E8E00C94792E6115710589F0DB010D903F
:105480000020E9F7AD0141505109461B570BDC01E3
:10549000ED91FC910280F381E02D0995089580E063
:1054A00090E00895EF92FF920F931F93CF93DF93B5
:1054B0008C01FB01C0E0D0E064917F018FEFE81A1E
:1054C000F80A662361F0D801ED91FC910190F0811A
:1054D000E02DC8010995C80FD91FF701EDCFCE0106
:1054E000CDB7DEB7E6E00C947B2E0E943B2A0895F0
:1054F000DC01ED91FC910190F081E02D099508957A
:105500000F931F93CF93DF93EC016DE00E94782AF5
:105510008C016AE0CE010E94782A800F911FDF91F2
:10552000CF911F910F9108950F931F93CF93DF9306
:10553000EC010E94522A8C01CE010E94802A800F29
:10554000911FDF91CF911F910F9108950F931F939A
:10555000CF93DF93EC010E943B2A8C01CE010E9485
:10556000802A800F911FDF91CF911F910F91089595
:105570000F931F93CF93DF93EC010E94782A8C0145
:10558000CE010E94802A800F911FDF91CF911F9141
:105590000F910895A1E2B0E0E0EDFAE20C94592EEB
:1055A0007C01C42EE52FCB01D22E19A221E02D15AE
:1055B00010F02AE0D22E8E010F5D1F4F8D2C912C02
:1055C000A12CB12C6C2D7E2FA50194010E94122ECE
:1055D0008C2DD29E80191124015011098A3010F4AB
:1055E000805D01C0895CF80180832115310541058A
:1055F000510521F0C22EE32FCA01E4CFB801C70143
:105600000E943B2AA196ECE00C94752EA0E0B0E03D
:10561000ECE0FBE20C945D2EEC016A017B012115AC
:10562000310541F4E881F9810190F081E02D642F8A
:1056300009951DC02A303105A9F477FF12C06DE22B
:105640000E94782A8C0144275527BA014C195D091C
:105650006E097F092AE0CE010E94CA2A800F911F9D
:1056600006C02AE0B701A601CE010E94CA2ACDB722
:10567000DEB7E8E00C94792E9A01AB01662757FD5E
:105680006095762F0E94062B08950F931F93CF935A
:10569000DF93EC019A01AB01662757FD6095762FE9
:1056A0000E94062B8C01CE010E94802A800F911F40
:1056B000DF91CF911F910F9108952115310549F484
:1056C000DC01ED91FC910190F081E02D642F0995B2
:1056D00008950E94CA2A08959A01462F50E060E07A
:1056E00070E00E945D2B08959A01AB0160E070E0CC
:1056F0000E945D2B08950F931F93CF93DF93EC01CE
:105700000E945D2B8C01CE010E94802A800F911F88
:10571000DF91CF911F910F9108950F931F93CF9316
:10572000DF93EC019A01AB0160E070E00E945D2B19
:105730008C01CE010E94802A800F911FDF91CF91B2
:105740001F910F9108950F931F93CF93DF93EC0157
:105750009A01462F50E060E070E00E945D2B8C01C2
:10576000CE010E94802A800F911FDF91CF911F915F
:105770000F910895FC0124853585F901E05CFF4F08
:1057800080819181F901EE5BFF4F20813181821B85
:10579000930B8F7399270895FC0184859585FC01EF
:1057A000E05CFF4F40815181FC01EE5BFF4F2081A7
:1057B00031814217530741F00190F081E02DE80F4D
:1057C000F91F808190E008958FEF9FEF0895FC010D
:1057D00084859585FC01E05CFF4F40815181FC018F
:1057E000EE5BFF4F208131814217530779F0A08192
:1057F000B181A80FB91F8C91208131812F5F3F4F5C
:105800002F7333273183208390E008958FEF9FEF2C
:105810000895FC0181A1882329F0A489B5898C9180
:1058200086FFFBCF11A20895CF93DF93FC0126855D
:105830003785D901A05CBF4F8D919C91119701963E
:105840008F739927E901CE5BDF4F48815981841717
:105850009507D9F30D90BC91A02DA20FB31F6C93A7
:10586000A685B785A05CBF4F11969C938E93A689A1
:10587000B7892C9181E090E0078C02C0880F991FB6
:105880000A94E2F7282B2C9381E081A30488F58900
:10589000E02D80818064808381E090E0DF91CF9172
:1058A000089508951F920F920FB60F9211242F930F
:1058B0003F934F938F939F93EF93FF938091C000FB
:1058C00082FD1CC04091C600809188069091890697
:1058D00001968F73992720918A0630918B06821743
:1058E000930771F0E0918806F0918906E85BF94F23
:1058F0004083909389068093880602C08091C600F9
:10590000FF91EF919F918F914F913F912F910F9028
:105910000FBE0F901F90189582EE95E00E94BA2B53
:10592000892B11F00E94512C08951F920F920FB6EF
:105930000F9211242F933F938F939F93EF93FF9395
:105940002091440630914506809146069091470685
:105950002817390731F48091C1008F7D8093C100F1
:1059600014C0E0914606F0914706EC5FF94F2081A4
:10597000809146069091470601968F7399279093E0
:105980004706809346062093C600FF91EF919F91B2
:105990008F913F912F910F900FBE0F901F901895F0
:1059A000A0E0B0E0E6EDFCE20C94592EFC0113827D
:1059B000128288EE93E0A0E0B0E084839583A68312
:1059C000B7838CEB93E091838083758764875787D7
:1059D0004687318B208B138B028BF58AE48AD78A1A
:1059E000C68AB18EA08E938E828E8F85848F888991
:1059F000858F8989868F8A89878F8B8980A3ECE040
:105A00000C94752ECF92DF92EF92FF92CF93DF939B
:105A1000EC016A017B01411581EE580761057105B2
:105A2000F9F0EC89FD8981E090E008A002C0880FC0
:105A3000991F0A94E2F7808360E079E08DE390E0BB
:105A4000A70196010E94122E2150310941095109E6
:105A50005695479537952795211580E1380798F099
:105A6000EC89FD89108260E874E88EE190E0A7017E
:105A700096010E94122E2150310941095109569573
:105A8000479537952795E889F9893083EA89FB8915
:105A9000208319A2EE89FF89408181E090E09C017A
:105AA0000C8C02C0220F331F0A94E2F7422B408372
:105AB000EE89FF8940819C010D8C02C0220F331FAB
:105AC0000A94E2F7422B4083EE89FF8940819C01D2
:105AD0000E8C02C0220F331F0A94E2F7422B408340
:105AE000EE89FF8920810F8C02C0880F991F0A94CC
:105AF000E2F7809582238083DF91CF91FF90EF9032
:105B0000DF90CF9008958F929F92AF92BF92CF92E5
:105B1000DF92EF92FF920F931F9381E08F9385E0C6
:105B20008F9387E08F9383E08F9384E08F93E6ECED
:105B30008E2E912CF2ECAF2EB12CA1ECCA2ED12CD2
:105B4000B0ECEB2EF12C04EC10E025EC30E044E05E
:105B500056E068E476E082EE95E00E94D02C0F904B
:105B60000F900F900F900F901F910F91FF90EF905B
:105B7000DF90CF90BF90AF909F908F9008950E943C
:105B800003290E946822CCE8DCE20E9406252097C7
:105B9000E1F30E948C2CF9CFA29FB001B39FC0010A
:105BA000A39F700D811D1124911DB29F700D811D49
:105BB0001124911D08950E94CC2DA59F900DB49F96
:105BC000900DA49F800D911D11240895B7FF0C9492
:105BD000DB2D0E94DB2D821B930B0895DB018F933D
:105BE0009F930E94DB2DBF91AF91A29F800D911DCD
:105BF000A39F900DB29F900D1124089597FB072E3F
:105C000016F4009407D077FD09D00E94902E07FC6F
:105C100005D03EF4909581959F4F089570956195BC
:105C20007F4F0895A1E21A2EAA1BBB1BFD010DC0D8
:105C3000AA1FBB1FEE1FFF1FA217B307E407F5073C
:105C400020F0A21BB30BE40BF50B661F771F881F18
:105C5000991F1A9469F760957095809590959B01AE
:105C6000AC01BD01CF010895052E97FB1EF40094F1
:105C70000E944B2E57FD07D00E94122E07FC03D026
:105C80004EF40C944B2E50954095309521953F4FF6
:105C90004F4F5F4F089590958095709561957F4F18
:105CA0008F4F9F4F08952F923F924F925F926F9226
:105CB0007F928F929F92AF92BF92CF92DF92EF929C
:105CC000FF920F931F93CF93DF93CDB7DEB7CA1B1D
:105CD000DB0B0FB6F894DEBF0FBECDBF09942A8848
:105CE000398848885F846E847D848C849B84AA84F0
:105CF000B984C884DF80EE80FD800C811B81AA817D
:105D0000B981CE0FD11D0FB6F894DEBF0FBECDBF47
:105D1000ED010895EE0FFF1F0590F491E02D099419
:105D2000AA1BBB1B51E107C0AA1FBB1FA617B707C1
:105D300010F0A61BB70B881F991F5A95A9F78095DD
:105D40009095BC01CD0108958F929F92AF92BF9222
:105D5000CF92DF92EF92FF92CF93DF93EC016881B5
:105D600079818A819B81611571058105910521F4F5
:105D700064E279ED8BE597E02DE133EF41E050E00F
:105D80000E94342E49015A019B01AC01A7EAB1E4FB
:105D90000E94DB2D6B017C01ACEEB4EFA5019401F8
:105DA0000E94E92DC60ED71EE81EF91EF7FE06C09A
:105DB00081E0C81AD108E10880E8F80AC882D982CF
:105DC000EA82FB82C701B6019F77DF91CF91FF90F6
:105DD000EF90DF90CF90BF90AF909F908F900895FD
:105DE0000E94A42E089586E091E00E94A42E0895BA
:105DF0006093060170930701809308019093090155
:105E000008952F923F925F926F927F928F929F920E
:105E1000AF92BF92CF92DF92EF92FF920F931F93B8
:105E2000CF93DF938B01EA016115710521F0DB014E
:105E30008C9311969C93209739F09E012250310942
:105E40002332310508F0D8C07C016701BFEFCB1ABF
:105E5000DB0A5601F7016080862D90E00E94333006
:105E6000892B11F07601F1CFFDE26F120AC05701C4
:105E700082E0A80EB11CD70111966C907724739420
:105E80000BC0BBE26B1207C05701E2E0AE0EB11CC3
:105E9000D70111966C90712CCE018F7E892B89F4DD
:105EA000B0E36B1237C0F50180818F7D8835D1F466
:105EB0006180F2E0AF0EB11C872D8260782EC0E1C8
:105EC000D0E0CA30D10551F1C031D10521F0C83040
:105ED000D10599F409C0CC24CA94DC2CEC2CAFE099
:105EE000FA2E22C0209769F7C8E0D0E0CC24CA94EB
:105EF000DC2CEC2CFFE1FF2E17C06FEF7FEFCB0106
:105F00009E01442737FD4095542F0E94122E6901AF
:105F10007A010AC02097A9F6CAE0D0E0E9E9CE2EBE
:105F2000DC2CEC2CE9E1FE2EF50160E020E030E015
:105F3000A9014E01AA2497FCA094BA2C1F0170ED70
:105F4000572E560CA9E0A51570F48FEB860D8A31FB
:105F500018F499EC592E06C08FE9860D8A3148F560
:105F600089EA582E560C852D90E08C179D070CF56C
:105F70006F3FD9F0C216D306E406F50698F0C501C6
:105F8000B4010E94EE2D9B01AC01852D90E0A0E0B4
:105F9000B0E0280F391F4A1F5B1F281739074A072F
:105FA0005B0710F46FEF01C061E03196D1016C9096
:105FB000C5CF0115110551F0662311F0319703C0CB
:105FC00071FE04C03297D801ED93FC9370FE07C0B8
:105FD00050954095309521953F4F4F4F5F4F67FF4C
:105FE00010C082E290E090938D0680938C066FEF54
:105FF0007FEF8FEF9FEF07C060E070E080E090E000
:1060000002C0B901CA01DF91CF911F910F91FF909A
:10601000EF90DF90CF90BF90AF909F908F907F9048
:106020006F905F903F902F900895FC0188279927EB
:10603000E89421912032E9F3293010F02E30C8F392
:106040002B3241F02D3239F4689404C00E9467303D
:10605000820F911D219120532A30C0F31EF4909598
:1060600081959F4F0895911150C0803219F0895049
:106070008550D0F7089548EC53E00E9440300895D1
:10608000FA01A191B081009719F41097E1F0CD01C8
:10609000DC01CD010D90002011F4C00113C0FB0103
:1060A0002191222319F02015D9F7F3CFFB0121917B
:1060B000201519F41E92119606C02223C1F70D90E7
:1060C0000020A1F7D001FA01A193B08308957AE0EE
:1060D000979F902D879F802D910D11240895F999F8
:1060E000FECF92BD81BDF89A992780B50895262FDD
:1060F000F999FECF1FBA92BD81BD20BD0FB6F894AD
:10610000FA9AF99A0FBE019608959927882708955B
:04611000F894FFCF31
:1061140000008E06200001000000FF0002000200C3
:10612400020002000200020002000200020002005B
:1061340002000200020002000200028025000005A5
:10614400400AA1204EA50020244EA52C2330C012C5
:1061540000001A400AA1204EA5001B1E27522C2322
:10616400308025000005400AA1204EA50020244EC1
:10617400A52C2330004B000006400AD0009D4900A6
:106184007B289D492C233000E1000005400A45018D
:10619400D7DC03B81E0EBF00232E48E801008A4056
:1061A4000A6001555502AD1E20000023C801545851
:1061B4002074696D656F75742100596573004E6FA5
:1061C400002C00386368004E2F41002C205B005DDA
:1061D4002028002900486F70206368616E6E656C2A
:1061E400200020402000456E746572696E6720614E
:1061F40064617074697665206368616E6E656C2095
:1062040073656C656374696F6E2C207069636B6968
:106214006E673A007363616E6E6572206D6F6465BC
:10622400004E4F5420454E41424C45440053656E48
:1062340064696E672073657474696E677320746F24
:106244002052580A00526573657474696E6720732E
:10625400657474696E6773206F6E2052580A00412A
:10626400626F727465642065646974730A00696E90
:1062740076616C69642073656C656374696F6E0024
:106284000D0A496E76616C696420696E70757420BC
:106294002D2064697363617264656421070053652A
:1062A4007474696E677320736176656420746F20FB
:1062B400454550524F4D0A005265766572746564C7
:1062C4002073657474696E67732066726F6D204500
:1062D4004550524F4D0A004C6F61646564206661FD
:1062E40063746F72792064656661756C74730A00F7
:1062F4004B657920616E64206368616E6E656C73B2
:106304002072616E646F6D697A65640A004F70650E
:106314006E4C52536E6720545820737461727469C2
:106324006E672000206F6E20485720006D6F6475E3
:106334006C65206C6F636B65643F00342B340038EC
:1063440000382B340031320031322B340031360026
:1063540050504D0052535349005344410053434C51
:1063640000525844005458440041494E004C4245A0
:1063740045500053504B54524D0053425553005313
:10638400554D44004C4C494E440000070B0C101171
:106394001500B7012B032F033103350338033D03E5
:1063A400B7014003440349034D0351035503590303
:1063B4005D0363036A036F0374038D028D028D0210
:1063C4008D02160A1322312900000000142C192A08
:0863D400BA2BE72BCC2B092C9E
:107E00000F92CDB7DEB7112484B714BE81FFF1D035
:107E100082E08093C00088E18093C10086E0809377
:107E2000C20080E18093C4008EE0CDD088249924E4
:107E3000CC24C394F5E0DF2EE1E1EE2E73E0F72EC3
:107E4000B6D0082F813479F4B2D08983C2D0898129
:107E5000823811F481E005C0813811F485E001C059
:107E600083E09ED09AC0823411F484E103C085344B
:107E700019F485E0B6D091C0853561F498D0082F0B
:107E800010E095D090E0982E8824802A912A880CC2
:107E9000991C82C0863521F484E0A3D080E0E1CF34
:107EA000843609F04CC083D082D0A82E80D0B82E62
:107EB00000E011E07CD0F80181938F01AE16D1F77C
:107EC00088D0FB2DF53489F4E0E0F1E00BC0F9999E
:107ED000FECF92BC81BC0894811C911C819180BD15
:107EE000FA9AF99AEA1598F358C08B2D863409F05E
:107EF00054C0F401F7BEE89507B600FCFDCFF401CD
:107F0000A0E0B1E02C9130E011968C91119790E0B7
:107F1000982F8827822B932B12960C01C7BEE895C9
:107F20001124329681E0A038B80761F7F401D7BE7A
:107F3000E89507B600FCFDCFE7BEE8952EC0843774
:107F4000F1F435D034D0182F32D0B82E42D0FB2DDA
:107F5000F63421F4F40105914F010CC0FB2DF534EA
:107F600049F4F999FECF92BC81BC0894811C911C04
:107F7000F89A00B5802F14D0115049F70EC08537FC
:107F800039F427D08EE10CD085E90AD08FE069CF93
:107F9000813511F488E017D01CD080E101D050CF9A
:107FA0009091C00095FFFCCF8093C600089580910A
:107FB000C00087FFFCCF8091C00084FD01C0A89560
:107FC0008091C6000895E0E6F0E098E19083808318
:107FD0000895EDDF803219F088E0F5DFFFCF84E10E
:107FE000DFCF1F93182FE3DF1150E9F7F2DF1F9166
:0E7FF0000895282E80E0E7DFEE27FF27099492
:027FFE0001057B
:0400000300007E007B
:00000001FF
